:0400000078EF21F084
:08000800056ED8CF06F0E0CF31
:1000100007F00001E9CF0DF0EACF08F0E1CF09F0D9
:10002000E2CF0AF0D9CF0BF0DACF0CF0F3CF14F017
:10003000F4CF15F0FACF16F000C00FF001C010F0A9
:1000400002C011F003C012F004C013F09DAA2CEFFF
:1000500000F09EBA20EF02F00FC000F010C001F0D7
:1000600011C002F012C003F013C004F00DC0E9FF8C
:1000700008C0EAFF088E09C0E1FF0AC0E2FF0BC01A
:10008000D9FF0CC0DAFF14C0F3FF15C0F4FF16C08F
:10009000FAFF055007C0E0FF06C0D8FF1000F2CFFE
:1000A0000EF0F29EF76AB80FF66E000EF722090006
:1000B000F5500EBEF28E1200501043D10052104582
:1000C000D300F2CF0EF0F29EF76ADC0FF66E000E50
:1000D000F7220900F5500EBEF28E1200000000005B
:1000E0000000F2CF0EF0F29EF76AFC0FF66E000EE3
:1000F000F7220900F5500EBEF28E1200511043CFC8
:100100000000F2CF0EF0F29E1A0FF66E010EF722EB
:100110000900F5500EBEF28E1200001083638000BD
:1001200056312E35000000000000000000000000E5
:1001300000000000000000000000000000000000BF
:100140000000011083460800466565646261636BC8
:1001500020696E20487A00000000000000000000C6
:100160000000000000000000000002108345810034
:1001700044656661756C74204E6F64652049442047
:10018000666F72204952000000000000000000006D
:10019000000003100345DC0054656D70204E6F6451
:1001A0006520494420666F7220495200000000001B
:1001B0000000000000000000000050100343D100C8
:1001C000706F73636F6D6D00000000000000000031
:1001D000000000000000000000000000000000001F
:1001E000000051100143CF0041637475616C2050D1
:1001F0006F7300000000000000000000000000001D
:100200000000000000000000000052100345D30071
:1002100043757272656E74207370656564000000CA
:1002200000000000000000000000000000000000CE
:10023000000014100146D900726177414443000068
:1002400000000000000000000000000000000000AE
:100250000000000000000000000015100145DB0058
:1002600063757272656E742053656E73650000006D
:10027000000000000000000000000000000000007E
:10028000000020108343020063616C6363656E7439
:10029000000000000000000000000000000000005E
:1002A0000000000000000000000021108346040050
:1002B00063616C63616D700000000000000000006D
:1002C000000000000000000000000000000000002E
:1002D0000000261083460C00496E697469616C2029
:1002E00053706565642061742073746172747570F5
:1002F00000000000000000000000271083430E00F3
:10030000496E697469616C20506F736974696F6EAE
:1003100000000000000000000000000000000000DD
:10032000000060100341D40063616C4D6F64650090
:1003300000000000000000000000000000000000BD
:100340000000000000000000000000180160C5006F
:10035000706F7366656564000000000000000000B7
:10036000000000000000000000000000000000008D
:100370000000001A01610000000000000000000001
:10038000000000000000000000000000000000006D
:1003900000000000000000000000001401604D009B
:1003A000706F73636F6D6D20504D49440000000005
:1003B000000000000000000000000000000000003D
:1003C00000000016016100000000000000000000B5
:1003D000000000000000000000000000000000001D
:1003E000000000000000000000000000000000000D
:1003F00000000000000000000000000000000000FD
:1004000000000000000000000000000000000000EC
:10041000000001015751016A565D03E256C100F028
:100420000CD0006A080E586F563700365751005CE2
:10043000D8B0006E0136582FF7D7000135EF02F023
:100440009EAA1ED0036A01010651010FE96E010E3A
:100450000320EA6E9EAAFED7AECFEFFF062B06C1A1
:1004600056F1030E576F0001D4D700C006F1010109
:10047000065305E101C104F102C105F10781000144
:100480009E9A2CEF00F0200E926E01012A6B2A51E9
:10049000080811E3036A2A51140F016E000E0322AB
:1004A00001500001FB25E96EFC510320EA6EEF6A62
:1004B00001012A2BECD7080E1A6E256E196A186AEC
:1004C000246A236A040E0001FB25E96E000EFC215C
:1004D000EA6EEF6A050EFB25E96E000EFC21EA6E5E
:1004E000EF6AB2EF21F0010EEA6E2E0EE96EEF50C8
:1004F0000DE0060E016E006A002EFED7012EFBD71E
:100500007B0E006E002EFED7EF2EF3D7000C0101FC
:1005100042514403F3CF01F0F4CF00F04503F35010
:10052000002643514403F3500020026E0001000CEA
:1005300001012D6B2E6B160E396F386B3C6B2C6BDB
:10054000436B2CC142F1456B280E446F0001DFDF85
:1005500002C03EF102C003F001010150F2CF3DF1B3
:10056000F29E02C0F7FF0001CCDD0900F5CF03F0D9
:1005700001013DBFF28E3D6F03C03EF13D5302E1EC
:100580003E532BE03C5329E1436B2CC142F1456BB8
:10059000280E446F0001BBDF02C03EF102C003F031
:1005A00001010150F2CF3DF1F29E02C0F7FF0001C0
:1005B000A8DD0900F5CF03F001013DBFF28E3A6FCF
:1005C00003C03BF138513A5D06E139513B5D03E12F
:1005D000010E3C6F01D02C2BB3D73CC101F001526E
:1005E00005E0010E2E6F220E2D6F02D02E6B2D6BAB
:1005F0002EC14EF02DC14DF0160E396F010E386F21
:100600003C6B2C6B436B2CC142F1456B280E446F45
:1006100000017DDF02C03EF102C003F00101015084
:10062000F2CF3DF1F29E02C0F7FF00016ADD090042
:10063000F5CF03F001013DBFF28E3D6F03C03EF1E7
:100640003D5302E13E532BE03C5329E1436B2CC167
:1006500042F1456B280E446F000159DF02C03EF1A4
:1006600002C003F001010150F2CF3DF1F29E02C041
:10067000F7FF000146DD0900F5CF03F001013DBFA2
:10068000F28E3A6F03C03BF138513A5D06E13951C1
:100690003B5D03E1010E3C6F01D02C2BB3D73CC175
:1006A00001F0015203E02E6B2D6B02D02E6B2D6BEF
:1006B0002EC150F02DC14FF0160E396F020E386F5B
:1006C0003C6B2C6B436B2CC142F1456B280E446F85
:1006D00000011DDF02C03EF102C003F00101015024
:1006E000F2CF3DF1F29E02C0F7FF00010ADD0900E2
:1006F000F5CF03F001013DBFF28E3D6F03C03EF127
:100700003D5302E13E532BE03C5329E1436B2CC1A6
:1007100042F1456B280E446F0001F9DE02C03EF144
:1007200002C003F001010150F2CF3DF1F29E02C080
:10073000F7FF0001E6DC0900F5CF03F001013DBF42
:10074000F28E3A6F03C03BF138513A5D06E1395100
:100750003B5D03E1010E3C6F01D02C2BB3D73CC1B4
:1007600001F0015203E02E6B2D6B02D02E6B2D6B2E
:100770002EC1C2F02DC1C1F0160E396F030E386FB5
:100780003C6B2C6B436B2CC142F1456B280E446FC4
:100790000001BDDE02C03EF102C003F001010150C4
:1007A000F2CF3DF1F29E02C0F7FF0001AADC090082
:1007B000F5CF03F001013DBFF28E3D6F03C03EF166
:1007C0003D5302E13E532BE03C5329E1436B2CC1E6
:1007D00042F1456B280E446F000199DE02C03EF1E4
:1007E00002C003F001010150F2CF3DF1F29E02C0C0
:1007F000F7FF000186DC0900F5CF03F001013DBFE2
:10080000F28E3A6F03C03BF138513A5D06E139513F
:100810003B5D03E1010E3C6F01D02C2BB3D73CC1F3
:1008200001F0015203E02E6B2D6B02D02E6B2D6B6D
:100830002EC1C4F02DC1C3F01A0E396F386B3C6B5A
:100840002C6B436B2CC142F1456B280E446F0001A9
:100850005EDE02C03EF102C003F001010150F2CFA2
:100860003DF1F29E02C0F7FF00014BDC0900F5CF1D
:1008700003F001013DBFF28E3D6F03C03EF13D53D9
:1008800002E13E532BE03C5329E1436B2CC142F182
:10089000456B280E446F00013ADE02C03EF102C0F3
:1008A00003F001010150F2CF3DF1F29E02C0F7FFCB
:1008B000000127DC0900F5CF03F001013DBFF28EF6
:1008C0003A6F03C03BF138513A5D06E139513B5D67
:1008D00003E1010E3C6F01D02C2BB3D73CC101F0DA
:1008E000015205E0020E2E6F220E2D6F02D02E6BEC
:1008F0002D6B2EC1C6F02DC1C5F01A0E396F010E39
:10090000386F3C6B2C6B436B2CC142F1456B280E4E
:10091000446F0001FCDD02C03EF102C003F00101A2
:100920000150F2CF3DF1F29E02C0F7FF000181ECD1
:1009300000F00900F5CF03F001013DBFF28E3D6FDD
:1009400003C03EF13D5302E13E532CE03C532AE10B
:10095000436B2CC142F1456B280E446F0001D7DD7B
:1009600002C03EF102C003F001010150F2CF3DF19F
:10097000F29E02C0F7FF000181EC00F00900F5CF04
:1009800003F001013DBFF28E3A6F03C03BF13851D5
:100990003A5D06E139513B5D03E1010E3C6F01D048
:1009A0002C2BB1D73CC101F0015203E02E6B2D6B13
:1009B00002D02E6B2D6B2EC1C8F02DC1C7F01A0EC0
:1009C000396F020E386F3C6B2C6B436B2CC142F1BC
:1009D000456B280E446F00019ADD02C03EF102C053
:1009E00003F001010150F2CF3DF1F29E02C0F7FF8A
:1009F000000181EC00F00900F5CF03F001013DBFDB
:100A0000F28E3D6F03C03EF13D5302E13E532CE0B8
:100A10003C532AE1436B2CC142F1456B280E446FD5
:100A2000000175DD02C03EF102C003F0010101507A
:100A3000F2CF3DF1F29E02C0F7FF000181EC00F021
:100A40000900F5CF03F001013DBFF28E3A6F03C0FC
:100A50003BF138513A5D06E139513B5D03E1010E4E
:100A60003C6F01D02C2BB1D73CC101F0015203E007
:100A70002E6B2D6B02D02E6B2D6B2EC1CAF02DC1AB
:100A8000C9F01A0E396F030E386F3C6B2C6B436B39
:100A90002CC142F1456B280E446F000138DD02C0C5
:100AA0003EF102C003F001010150F2CF3DF1F29E90
:100AB00002C0F7FF000181EC00F00900F5CF03F060
:100AC00001013DBFF28E3D6F03C03EF13D5302E197
:100AD0003E532CE03C532AE1436B2CC142F1456B61
:100AE000280E446F000113DD02C03EF102C003F086
:100AF00001010150F2CF3DF1F29E02C0F7FF00016B
:100B000081EC00F00900F5CF03F001013DBFF28E4A
:100B10003A6F03C03BF138513A5D06E139513B5D14
:100B200003E1010E3C6F01D02C2BB1D73CC101F089
:100B3000015203E02E6B2D6B02D02E6B2D6B2EC15C
:100B4000CCF02DC1CBF0000195EF0AF00101476B0D
:100B50004651475D25E247514525486F036A475195
:100B60004325E96E44510320EA6EEFCF49F1AA6AAA
:100B700048C1A9FF49C1A8FFA69CA69EA684F2CFA2
:100B800000F0F29E0F01550EA76EAA0EA76EA68268
:100B9000A6B2FED7A6940050F2120101472BD8D777
:100BA0000001000C230E01012F6F290E2E6F010E84
:100BB000446F2E0E436F0E0E456F020E466F0001FE
:100BC000C5DF01012D6BFF0E2C6F010E446F2C0E43
:100BD000436F0C0E456F020E466F0001B7DF010137
:100BE0002D6B0A0E2C6F010E446F2C0E436F080EF6
:100BF000456F020E466F0001A9DF01012F6B2E6BBE
:100C0000010E446F2C0E436F020E456F466F0001BC
:100C10009DDF230E01012F6F280E2E6F010E446FF2
:100C20002E0E436F040E456F020E466F00018EDFDD
:100C300097EF0AF001013251080804E0336F3137B1
:100C4000332FFDD79488949A94968B9693908A909C
:100C500032C133F131AF8B9A31BF8B8A31378B86FA
:100C6000013682A8019082B801808B96332FF2D78B
:100C70008A808A900001EDEF06F001012F6B306B46
:100C8000010E0001FB25E96E000EFC21EA6EEF5219
:100C90000BE1050EFB25E96E000EFC21EA6EEF6A02
:100CA00001012F6B94D00001050EFB25E96E000EAB
:100CB000FC21EA6EEFCF31F1090EFB25E96E000E43
:100CC000FC21EA6E040EEF240101315D08E1050EFE
:100CD0000001FB25E96E000EFC21EA6EEF6A050EAD
:100CE0000001FB25E96E000EFC21EA6EEFCF31F129
:100CF000090EFB25E96E000EFC21EA6E030EEF24BF
:100D00000101315D0AE1440E2F6F010E0001FB2548
:100D1000E96E000EFC21EA6EEF6A050E0001FB256C
:100D2000E96E000EFC21EA6EEFCF31F1090EFB25D2
:100D3000E96E000EFC21EA6E030EEF240101315D25
:100D40002AE2050E0001FB25E96E000EFC21EA6E89
:100D5000EF52D8A402D001011ED0050EFB25E96E8A
:100D6000000EFC21EA6E010EEF5C036A140F016EA7
:100D7000000E03220150FB25E96EFC510320EA6EB0
:100D8000EFCF2FF10101050E0001FB25E96E000EEA
:100D9000FC21EA6EEF2A050E0001FB25E96E000E2C
:100DA000FC21EA6EEF5212E1090EFB25E96E000EFE
:100DB000FC21EA6EEF50B00901012F6F050E000112
:100DC000FB25E96E000EFC21EA6EEF2A01012FC11E
:100DD00031F1080E326F00012DD7015001C030F102
:100DE000FBC0E9FFFCC0EAFFEF6A040EFB25E96ED9
:100DF000000EFC21EA6EEFCF31F1080EFB25E96E03
:100E0000000EFC21EA6E040EEF240101315D08E1C1
:100E1000040E0001FB25E96E000EFC21EA6EEF6A6C
:100E2000040E0001FB25E96E000EFC21EA6EEFCFF7
:100E300031F1080EFB25E96E000EFC21EA6E030E6F
:100E4000EF240101315D1BE13051440810E1000144
:100E5000FBC0E9FFFCC0EAFF010EEF6E040EFB25AC
:100E6000E96E000EFC21EA6EEF2A09D00101040EA2
:100E70000001FB25E96E000EFC21EA6EEF6A040E0C
:100E80000001FB25E96E000EFC21EA6EEFCF31F187
:100E9000080EFB25E96E000EFC21EA6E030EEF241E
:100EA0000101315D28E2040E0001FB25E96E000E10
:100EB000FC21EA6EEF52D8A402D001011CD0040E2E
:100EC000FB25E96E000EFC21EA6E010EEF5C036A61
:100ED0000A0F016E000E03220150FB25E96EFC5142
:100EE0000320EA6E30C1EFFF040EFB25E96E000E11
:100EF000FC21EA6EEF2A040E0001FB25E96E000ECC
:100F0000FC21EA6EEF5222E101013051F00BB008F2
:100F100015E1080E0001FB25E96E000EFC21EA6ECA
:100F2000010130510F0BEF6E040E0001FB25E96E3D
:100F3000000EFC21EA6EEF2A09D00101040E000127
:100F4000FB25E96E000EFC21EA6EEF6A4EEF09F018
:100F500001014C3D2DD04B31036E4A31026E4931B7
:100F6000016E4831006E0332023201320032033228
:100F70000232013200321F0E031600C04DF146C18D
:100F8000E9FF47C1EAFF4DC1EFFF4851070B4D6F25
:100F9000010E4625016E000E472101C0E9FFEA6EF1
:100FA0004D39006E0036E00E001600C0EFFF5AD03B
:100FB00047C103F046C1E9FF47C1EAFF4B31016E6B
:100FC0004A31006E01320032013200320132003209
:100FD00001320032070E011600C0EFFF010E462558
:100FE000016E000E4721036E01C0E9FFEA6E4B312E
:100FF000536F4A31526F4931516F5333523351332A
:1010000053335233513353335233513353335233B7
:101010005133070E53175151E00BEF6E010E462569
:10102000016E000E4721036E01C0E9FFEA6E4A51CE
:10103000030B006E0050EF10EF6E020E4625016E9E
:10104000000E4721036E01C0E9FFEA6E49C1EFFFC0
:10105000030E4625016E000E472101C0E9FFEA6E2E
:1010600048C1EFFF0001000C0F0140B757D001014C
:101070004053D8B402D00F0151D0F00E6F166F86D6
:101080004451030B0F014013010144B710D00F0E60
:10109000476F410E466F4B6B4A6B3FC149F13EC1F2
:1010A00048F1F70E4C6F000153DF0FD001010F0E16
:1010B000476F410E466F4B6B4A6B3FC149F13EC1D2
:1010C00048F1FF0E4C6F000143DF43C145FF0101B2
:1010D00044BD03D00F01458D0101456B4351455D72
:1010E0001AE2460E4525016E0F0E036ED8B0032A94
:1010F00003C047F1036A45514125E96E425103207F
:10110000EA6EEFCF48F147C1EAFF01C0E9FF48C1ED
:10111000EFFF452BE3D70F014087B7D030B758D04A
:101120000101402D01D002D00F0152D0F00E6F16F8
:10113000060E6F124451030B0F013013010144B727
:1011400010D00F0E476F310E466F4B6B4A6B3FC18D
:1011500049F13EC148F1F70E4C6F0001F9DE0FD0A6
:1011600001010F0E476F310E466F4B6B4A6B3FC14B
:1011700049F13EC148F1FF0E4C6F0001E9DE43C169
:1011800035FF010144BD03D00F01358D0101456BD1
:101190004351455D1AE2360E4525016E0F0E036E72
:1011A000D8B0032A03C047F1036A45514125E96ECF
:1011B00042510320EA6EEFCF48F147C1EAFF01C078
:1011C000E9FF48C1EFFF452BE3D70F0130875DD022
:1011D00020B758D0010140510208D8B402D00F0105
:1011E00051D0F00E6F166F844451030B0F01201382
:1011F000010144B710D00F0E476F210E466F4B6BA5
:101200004A6B3FC149F13EC148F1F70E4C6F0001F6
:101210009FDE0FD001010F0E476F210E466F4B6B03
:101220004A6B3FC149F13EC148F1FF0E4C6F0001CE
:101230008FDE43C125FF010144BD03D00F01258D81
:101240000101456B4351455D1AE2260E4525016EAD
:101250000F0E036ED8B0032A03C047F1036A45514D
:101260004125E96E42510320EA6EEFCF48F147C1B4
:10127000EAFF01C0E9FF48C1EFFF452BE3D70F01AB
:10128000208703D0000E016E03D06F6A010E016E3D
:101290000001000C01012E6B0001EFD4FBC0E9FF3F
:1012A000FCC0EAFFEF2C7AD00B0EFB25E96E000E96
:1012B000FC21EA6EEF5272E00A0EFB25E96E000E89
:1012C000FC21EA6EEF500101306B2F6F306F2F6BF6
:1012D0000B0E0001FB25E96E000EFC21EA6EEF50BB
:1012E000036A01012F11186E03503011196E0B0E95
:1012F0000001FB25E96E000EFC21EA6EEFCF4CF0F9
:10130000080EFB25E96E000EFC21EA6EEFCF1AF005
:10131000020E01012E6F080E0001FB25E96E000E82
:10132000FC21EA6E020EEF2401012E5D28E2020E7E
:101330002E5D036A030F016E000E03220150180F89
:10134000016E000E032201C02FF103C030F1036AC9
:101350002E510A0F016E000E032201500001FB25E1
:10136000E96EFC510320EA6EEFCF31F1010130C18B
:10137000EAFF2FC1E9FF31C1EFFF2E2BCCD719C0F7
:101380003FF118C03EF1020E406F426B1B0E416FE1
:101390001AC043F1FC0E446F000166DE000C140E0F
:1013A000FB25E96E000EFC21EA6EEF6A150EFB25A7
:1013B000E96E000EFC21EA6EEF6A090EFB25E96E6C
:1013C000000EFC21EA6E020EEF6E160EFB25E96E92
:1013D000000EFC21EA6E810EEF6E170EFB25E96E02
:1013E000000EFC21EA6EEF6A010EFB25E96E000E8D
:1013F000FC21EA6E010EEF6E01012D6B2D511308D9
:101400000BE3000147DF140E01012E6F000173ECA6
:1014100002F001012D2BF2D7000167EF0AF0140E44
:10142000FB25E96E000EFC21EA6E060EEF6E150E2E
:10143000FB25E96E000EFC21EA6EEF6A090EFB2522
:10144000E96E000EFC21EA6E050EEF6E160EFB250E
:10145000E96E000EFC21EA6E200EEF6E170EFB25E2
:10146000E96E000EFC21EA6E010EEF6E180EFB25F0
:10147000E96E000EFC21EA6EEF6A190EFB25E96E9B
:10148000000EFC21EA6E100EEF6E1A0EFB25E96EBF
:10149000000EFC21EA6E4CC0EFFF010EFB25E96E49
:1014A000000EFC21EA6E010EEF6E01012C6B2C5137
:1014B00013080BE30001EEDE140E01012E6F000194
:1014C00073EC02F001012C2BF2D7000168D7E2EF98
:1014D0000AF0F2CF2CF1F29EAA6A800EA96EA69CA9
:1014E000A69EA680A85001012CBFF28E4B6E4B52D7
:1014F00003E04B50FD081CE2AA6A800EA96E220E82
:10150000A86EA69CA69EA684F2CF00F0F29E0F01C4
:10151000550EA76EAA0EA76EA682A6B2FED7A694F7
:101520000050F212000198EF02F0D2EF05F0010135
:10153000F2CF2CF1F29EAA6A800EA96EA69CA69EFE
:10154000A680A8502CBFF28E4B6EF2CF2CF1F29EEB
:10155000AA6A810EA96EA69CA69EA680A8502CBF42
:10156000F28E4C6E4C5203E04C50FD081CE2AA6A0D
:10157000810EA96EA86AA69CA69EA684F2CF00F052
:10158000F29E0F01550EA76EAA0EA76EA682A6B2F6
:10159000FED7A6940050F212C80E01012E6F000172
:1015A00073EC02F00101F2CF2CF1F29EAA6A810ED7
:1015B000A96EA69CA69EA680A8502CBFF28E4C6E4B
:1015C00000012DD7036A4BC032F0070E0324336E9F
:1015D000060E346E050E356E91EF0EF035C16FFFBD
:1015E0006E50E00B0101355DD8B402D00001F8D790
:1015F0000001000C010135073607370738073907A6
:101600003539706E70367036C00E701636517012E5
:101610003735716E71367136F80E71163951711297
:101620003AB501D0718C3AA101D0718E38C172FFE8
:10163000728C000190EF0BF00101355305E10F0EA4
:101640003C6F180E3B6F04D00F0E3C6F1C0E3B6FAF
:101650003CC147F13BC146F139C14BF138C14AF1B8
:1016600037C149F136C148F13AC14CF1000170DC93
:10167000000C01013551000109E0010A0CE0030AE8
:1016800010E0010A14E0070A18E01DD00F0E010156
:101690003C6F3B6B1ED00F0E01013C6F040E3B6F85
:1016A00018D00F0E01013C6F080E3B6F12D00F0EC9
:1016B00001013C6F0C0E3B6F0CD00F0E01013C6F13
:1016C000100E3B6F06D00F0E01013C6F140E3B6FE6
:1016D00000D03CC147F13BC146F139C14BF138C1A3
:1016E0004AF137C149F136C148F13AC14CF1000124
:1016F0002FDC000C9350FB0B0809936E800E010148
:10170000356F00016BDF2DC135F12EC136F12FC1D0
:1017100037F130C138F131C139F132C13AF16AD70C
:1017200001013251600B606E32A901D0608460CF3C
:1017300050FF738A356B396B386B376B366BFF0E26
:101740003A6F000179DF010E0101356F396B386B9B
:10175000376B366BFF0E3A6F00016EDF01013251BD
:10176000600B9F09DF0A000103E0600A06E00AD06F
:10177000F70E0101336F346F0BD0FF0E0101336F91
:10178000346F06D0FF0E0101336FF70E346F00D0B7
:10179000356B396B386B376B366B33C13AF10001FF
:1017A00068DF010E0101356F396B386B376B366BB3
:1017B00033C13AF100015DDF020E0101356F396B73
:1017C000386B376B366B34C13AF1000152DF030ED0
:1017D0000101356F396B386B376B366B34C13AF1B9
:1017E000000147DF040E0101356F396B386B376B31
:1017F000366B34C13AF100013CDF050E0101356F53
:10180000396B386B376B366B34C13AF1000131DF1D
:101810000101356B0001E2DE1CEF0CF0010E01014D
:101820002D6F020E2E6F060E2F6F306F070E316F69
:10183000BF0E326F00015ED7800E0101356F0001CF
:10184000CDDE0101356B396B386B070E376FFF0E3C
:10185000366F3A6F0001F0DE4BC02DF10101060E2C
:10186000356B396B386B376F4BC036F1FF0E3A6F03
:101870000001FFDE010E0101356F396B386B376BEC
:10188000366BFF0E3A6F0001F4DE010E0101356F79
:10189000396B386B070E376FFF0E366F3A6F0001EA
:1018A000CBDE4BC04DF0010E4E6E4BC04FF0030E21
:1018B000506EC26BC16B4EC08BF04DC08AF050C0F1
:1018C00096F04FC095F0C2C0A1F0C1C0A0F0020ECA
:1018D0000101356F396B386B4EC037F14DC036F1B1
:1018E000FF0E3A6F0001C5DE030E0101356F396B43
:1018F000386B50C037F14FC036F1FF0E3A6F000120
:10190000B8DE040E0101356F396B386BC2C037F198
:10191000C1C036F1FF0E3A6F0001ABDE4CC02DF1B5
:101920000101060E2E6F050E356F396B386B2EC117
:1019300037F14CC036F1FF0E3A6F00019ADE4BC012
:10194000C5F0020EC66FC86BC76BCA6BC96BCC6B98
:10195000CB6BC6C05FF0C5C05EF0C8C06AF0C7C040
:1019600069F0CAC075F0C9C074F0CCC080F0CBC0BB
:101970007FF00101356B000131DE01012C6B2C5130
:1019800003080AE3036A2C512E0FE96E000E0320B0
:10199000EA6EEF6A2C2BF3D74A6A496A486A00015B
:1019A000D5EF0CF0870ED56E39D792EF0EF001010E
:1019B000456B4451455D19E2036A45514125E96E85
:1019C00042510320EA6E45514325486FF2CF49F159
:1019D000F29EAA6A48C1A9FFA69CA69EA680A8500E
:1019E00049BFF28EEF6E452BE4D70001000C8E0E3E
:1019F000006E2DC101F02CC102F0036A01AE05D0CA
:101A0000011E021E022A01E1012A015209E102C05F
:101A100001F0026A080E005E015202E1006A0DD078
:101A2000D89001BE04D0023601360006F9D7010174
:101A30002DAF02D0000101D0019E0001000C010178
:101A40003051D8B4A5D03C6F3451D8B4A1D03C5F4C
:101A500005E37F0E3C27D8B09BD006D0810E3C5FBB
:101A6000D8A096D0D8B494D03CC100F0016A026AE4
:101A7000036A3B6B31C13AF13A8F32C139F133C15C
:101A800038F1190E3C6F3751385F0DE2010E395FA6
:101A90000AE23A5F08E23B5F06E23B2B3A2B392B26
:101AA0003751382728D03651395F12E2010E3A5F9C
:101AB0000FE23B5F0DE23B2B3A2B36513927375172
:101AC000382719E3392B17E13A2B15E13B2B13D0BB
:101AD000355180093A5F0EE2010E3B5F0BE23B2B72
:101AE000355180093A2736513927E9E33A2BE7E1A6
:101AF0003B2BE5D703803C2F01D00BD0D890383753
:101B000039373A373B37D8900336023601363D37FE
:101B1000BAD73DA106D0D8900132023203323D330C
:101B200002D0000635E03DBF1ED0D8903837393797
:101B30003A373B373751385F07E2010E395F04E22D
:101B40003A5F02E23B5F1AE33651395F05E2010E6C
:101B50003A5F02E23B5F12E3355180093A5F03E2EC
:101B6000010E3B5F0BE3032A09E1022A07E1012A88
:101B700005E1002A0DE001320232033231C13CF1AD
:101B800035513C1B3CAF02D0018E06D0019E04D0E3
:101B9000006A016A026A036A000137EF0EF0016A07
:101BA000026A006A036A01012F5102E12E5118E016
:101BB000100E306FD8902C372D37003603362F514A
:101BC000035C02E12E51005C07E32E51005ED8A0B9
:101BD00003062F51035ED88001360236302FEAD734
:101BE000000167EF0EF0D46B010E0101426F190E78
:101BF000416F0C0E436F020E446F0001D8DE0101ED
:101C000019C11BF11BC1D3F0010E426F130E416FBE
:101C1000020E436F446F0001CADE010E0101426FE4
:101C2000150E416F040E436F020E446F0001BFDEBC
:101C300016C12DF115C12CF1DADE00C02CF101C066
:101C40002DF102C02EF103C02FF103C033F102C009
:101C500032F101C031F100C030F10101376BA00E4B
:101C6000366F0C0E356F8C0E346F0001E8D603C052
:101C700012F102C011F101C010F100C00FF1010E0C
:101C80000101426F170E416F0E0E436F020E446F3B
:101C900000018DDE18C1D2F017C1D1F00101426BF5
:101CA000CD0E416F080E436F020E446F00017FDEC0
:101CB000CD5302E1CE530FE04C0E01012D6F470EC4
:101CC0002C6FCEC02FF1CDC02EF1000168D702C01D
:101CD000D8F001C0D7F0C150C00B0E09C16EC05082
:101CE000C00B0709C06EC08EC280000E016EC250CC
:101CF000C30B0110C26E93EF0EF0AB98AC9AC00EFE
:101D000094129D8AF212A0EF0EF0F29CF29EF2BEA7
:101D1000FDD7640E01012E6F000173EC02F069EF34
:101D20000AF040D660D7080E01012C6FFA0E2E6F14
:101D3000000173EC02F001012C2FF8D70001DDD770
:101D4000080E01012C6FFA0E2E6F000173EC02F0E9
:101D500001012C2FF8D7959E8C7E0001000C9EA8C7
:101D6000FED701012C51AD6EACA2FED7AD0E006EB8
:101D7000002EFED70001000CD65001010B6FD7CF0B
:101D80000CF107B119D0D650D7CF03F02A6FD7CFB7
:101D90002BF10B512A5F0C512B5B0E512B5D0BE38A
:101DA00003E12A510D5D07E2959A8C9A959C8C9CD3
:101DB000959E8C9E01D0E5D7000100EF0FF0010148
:101DC0000791650E086F0851FF0A010F086FAB9865
:101DD000AC8A800E2C6F0001C2DFE50E01012C6F72
:101DE0000001BDDF01012C6B0001B9DF01012C6B8B
:101DF0000001B5DF08C12CF1B2DFAB88AC9ABCD7CB
:101E000004C1FFF005C100F104C103F0010105C1E7
:101E100001F004C102F00001000C01013E5100017B
:101E200007E0010A09E0030A0AE0010A0BE00DD00D
:101E3000010E01013F6F0CD001013F6B09D0010180
:101E40003F6B06D001013F6B03D001013F6B00D017
:101E50003FC101F00001000C01012E51FC0F65E2B1
:101E6000040F00019AEF0FF001012F51050DF350FF
:101E7000326B316F020E3125016E000E3221036E7E
:101E80000150F2CF31F1F29E000171EC00F001013E
:101E900031BFF28E306F49D001012F51050DF35043
:101EA000326B316F020E3125016E000E3221036E4E
:101EB0000150F2CF31F1F29E000161EC00F001011E
:101EC00031BFF28E306F31D001012F51050DF3502B
:101ED000326B316F020E3125016E000E3221036E1E
:101EE0000150F2CF31F1F29E000161EC00F00101EE
:101EF00031BFF28E306F19D001012F51050DF35013
:101F0000326B316F020E3125016E000E3221036EED
:101F10000150F2CF31F1F29E000161EC00F00101BD
:101F200031BFF28E306F01D0010130C101F00001EC
:101F300071EF10F0F2CF0EF0F29EE824F76AF73658
:101F4000590FF66E1F0EF7220A00F550FA6E0800C0
:101F5000F5500EBEF28EF96E681E981EC81EF81E51
:101F600001013051FC0F79E2040F000134EF10F051
:101F700001013151050DF350356B346F030E3425DB
:101F8000016E000E3521036E0150F2CF34F1F29E46
:101F9000000171EC00F00900F5CF03F0010134BF3E
:101FA000F28E326F03C033F158D001013151050D6B
:101FB000F350356B346F030E3425016E000E35215E
:101FC000036E0150F2CF34F1F29E000161EC00F09B
:101FD0000900F5CF03F0010134BFF28E326F03C068
:101FE00033F13BD001013151050DF350356B346FA6
:101FF000030E3425016E000E3521036E0150F2CF21
:1020000034F1F29E000161EC00F00900F5CF03F01D
:10201000010134BFF28E326F03C033F11ED00101D3
:102020003151050DF350356B346F030E3425016EBD
:10203000000E3521036E0150F2CF34F1F29E000103
:1020400061EC00F00900F5CF03F0010134BFF28E1E
:10205000326F03C033F101D0010132C101F033C14D
:1020600002F00001A0EF10F0F2CF0EF0F29EE82493
:10207000F76AF7368D0FF66E200EF7220A00F5503C
:10208000FA6E0800F5500EBEF28EF96E701FAA1F90
:10209000E41F1E2035500508D8A4C2D12AC13EF144
:1020A000BCDE01C02BF101012A510B0DF3502F6B47
:1020B0002E6F020E2E25016E000E2F21036E015091
:1020C0005E0FE96E000E0320EA6EEF6A2C6B2B5157
:1020D0002C5DD8B09CD12AC12EF12CC12FF100016A
:1020E000BBD601C02DF101012A510B0DF3502F6B0E
:1020F0002E6F030E2E27000E2F232A510B0DF350A7
:10210000316B306F020E3025016E000E3121036EEF
:1021100001505E0FE96E000E0320EA6E036AEF5075
:102120002E25016E2F51032201505E0F2E6F000EDF
:1021300003202F6F2AC130F12CC131F1000110D7DB
:1021400002C031F101C030F12DC143F10101435111
:10215000410A000113E0030A15E0010A17E0070A2B
:1021600019E0010A1BE0030A1DE0010A1FE00F0A43
:1021700021E02B0A23E0030A25E028D0010E016E9E
:102180002BD02AD0010E016E27D026D0020E016E70
:1021900023D022D0040E016E1FD01ED0010E016E7E
:1021A0001BD01AD0020E016E17D016D0040E016E8D
:1021B00013D012D0040E016E0FD00ED0010E016E9E
:1021C0000BD00AD0020E016E07D006D0AA0E486EC0
:1021D000000E016E01D000D001C032F12FC1EAFF24
:1021E0002EC1E9FF31C1E2FF30C1E1FF0101015021
:1021F000016E04E0E6CFEEFF012EFCD72D5148081A
:10220000D8A49AD02A510B0DF3502F6B2E6F030ECA
:102210002E27000E2F232A510B0DF350316B306FF8
:10222000020E3025016E000E3121036E01505E0F4B
:10223000E96E000E0320EA6E036AEF502E25016E50
:102240002F51032201505E0F2E6F000E03202F6FBF
:102250002FC141F12EC140F1010E4025436F000E08
:102260004121446F44C1EAFF43C1E9FFD890EF36F2
:10227000426BD8B0422B40C143F141C144F14253BB
:1022800002E1D89001D0D88044C1EAFF43C1E9FF00
:10229000ED32426BD8B0422B010E4025436F000E49
:1022A0004121446F425302E1D89001D0D88044C10B
:1022B000EAFF43C1E9FFED3240C1E9FF41C1EAFF56
:1022C000EFCF42F1030E4025E96E000E4121EA6E88
:1022D000EFCF45F141C1EAFF40C1E9FF45C1EFFF42
:1022E000030E4025E96E000E4121EA6E42C1EFFF68
:1022F000010E4025E96E000E4121EA6EEFCF42F15A
:10230000010E4025016E000E4121036E020E402594
:10231000E96E000E4121EA6EEFCF45F103C0EAFFFE
:1023200001C0E9FF45C1EFFF020E4025E96E000E36
:102330004121EA6E42C1EFFF2A510B0DF3502F6B82
:102340002E6F020E2E25016E000E2F21036E0150FE
:102350005E0F016E000E032201502E6F03C02FF19D
:102360002FC1EAFF2EC1E9FFEFCF30F12DC143F1BC
:102370004351410A000113E0030A15E0010A17E086
:10238000070A19E0010A1BE0030A1DE0010A1FE029
:102390000F0A21E02B0A23E0030A25E028D0010ED2
:1023A000016E2BD02AD0010E016E27D026D0020E4E
:1023B000016E23D022D0040E016E1FD01ED0010E5C
:1023C000016E1BD01AD0020E016E17D016D0040E6B
:1023D000016E13D012D0040E016E0FD00ED0010E7C
:1023E000016E0BD00AD0020E016E07D006D0AA0EE5
:1023F000486E000E016E01D000D001500101302561
:102400002FC1EAFF2EC1E9FFEF6E2C2B60D6036AC5
:102410002A512E0FE96E000E0320EA6E010EEF6EB8
:10242000000131EF12F0CBDC02C0DAF001C0D9F0CC
:10243000DAC043F1D9C042F10101456B0A0E446F85
:10244000000187EC02F0A40E0101015C006E380E61
:10245000025800C0CFF00001D06F01012A6B0001CB
:1024600019D6DEEF21F0010132C1E9FF33C1EAFFE5
:10247000EF6A60AEA5D0F00E6F163581A49074AEF1
:1024800008D032C1E9FF33C1EAFFEF500809EF6E0F
:10249000749E60A411D033C103F032C1E9FF33C18F
:1024A000EAFFEFCF00F000C0EFFF32C1E9FF33C118
:1024B000EAFFEF50010BEF6E30C1E9FF31C1EAFFD7
:1024C00065500F0BEF6E65AC07D032C1E9FF33C129
:1024D000EAFFEF504009EF6E62A608D032C1E9FF73
:1024E00033C1EAFFEF502009EF6E35D02CC1E9FF70
:1024F0002DC1EAFF3B6B3A6B396B6134006E3935A5
:10250000016E3A35026E3B35036E003601360236F7
:1025100003360036013602360336F80E001600C0C8
:10252000EFFF01C0ECFF2DC103F02CC1E9FF2DC16D
:10253000EAFF6250E00B006E003A0032070E001610
:102540000050016A0050EF10006E0150EC10ED5287
:1025500000C0EFFFEC6E346B31C103F030C1E9FF16
:1025600031C1EAFFEF50345D1FE2036A34512E257A
:10257000016E2F51032201C036F103C037F1660E00
:102580003425016E0F0E036ED8B0032A01C0E9FF97
:1025900003C0EAFFEFCF38F137C1EAFF36C1E9FFE8
:1025A00038C1EFFF342BD8D76F6AA4AE08D032C140
:1025B000E9FF33C1EAFFEF501009EF6EA49EC2D0CD
:1025C0000F0150AFBBD0F00E6F160A0E6F12010153
:1025D0003591A49274AC08D032C1E9FF33C1EAFF4F
:1025E000EF500809EF6E749C33C103F032C1E9FF6C
:1025F00033C1EAFFEFCF00F000C0EFFF33C103F0BB
:1026000032C1E9FF33C1EAFFEF50010807E332C1ED
:10261000E9FF33C1EAFFEF508009EF6E30C1E9FFF7
:1026200031C1EAFF0F0155510F0BEF6E55AD09D0C7
:10263000010132C1E9FF33C1EAFFEF504009EF6EFB
:102640000F0152A70AD0010132C1E9FF33C1EAFFED
:10265000EF502009EF6E3BD00F0101012CC1E9FFC3
:102660002DC1EAFF3B6B3A6B396B51CF38F13835EE
:10267000006E3935016E3A35026E3B35036E003619
:102680000136023603360036013602360336F80EBE
:10269000001600C0EFFF01C0ECFF2DC103F02CC1FC
:1026A000E9FF2DC1EAFF0F015251E00B006E003A25
:1026B0000032070E00160050016A0050EF10006E45
:1026C0000150EC10ED5200C0EFFFEC6E0101346BD5
:1026D00031C103F030C1E9FF31C1EAFFEF50345D91
:1026E0001FE2036A34512E25016E2F51032201C0CF
:1026F00036F103C037F1560E3425016E0F0E036E0E
:10270000D8B0032A01C0E9FF03C0EAFFEFCF38F1D8
:1027100037C1EAFF36C1E9FF38C1EFFF342BD8D704
:102720006F6AA4AE08D032C1E9FF33C1EAFFEF50AF
:102730001009EF6EA49E0F01509F03D0000E016E92
:102740000BD0010135A102D0609E03D00F01509F34
:102750000101010E016E0F01000184EF1EF0B7C0F0
:102760003FF1B6C03EF1020E0101406F426BB90E5F
:10277000416FB8C043F1FC0E446F000134EC08F027
:10278000015203E1AD0E486EEAD7486A000C010120
:102790003F51000107E0010A09E0030A0AE0010ACB
:1027A0000BE00DD0010E0101406F0CD00101406B18
:1027B00009D00101406B06D00101406B03D001013B
:1027C000406B00D040C101F00001000C01013F51FD
:1027D000FC0F69E2040F00015AEF14F001014051AF
:1027E000050DF350446B436F44C103F04351F2CFE6
:1027F00043F1F29E00014FEC00F00900F5CF03F029
:10280000010143BFF28E416F03C042F14CD0010180
:102810004051050DF350446B436F44C103F04351E5
:10282000F2CF43F1F29E000161EC00F00900F5CF18
:1028300003F0010143BFF28E416F03C042F133D078
:1028400001014051050DF350446B436F44C103F047
:102850004351F2CF43F1F29E000161EC00F0090018
:10286000F5CF03F0010143BFF28E416F03C042F187
:102870001AD001014051050DF350446B436F44C120
:1028800003F04351F2CF43F1F29E000161EC00F0FE
:102890000900F5CF03F0010143BFF28E416F03C081
:1028A00042F101D0010141C101F042C102F0000139
:1028B00029EF15F0F2CF0EF0F29EE824F76AF73612
:1028C000D90FF66E280EF7220A00F550FA6E0800AE
:1028D000F5500EBEF28EF96EDC270E2840287228C5
:1028E00001013F51FC0F69E2040F0001E4EF14F015
:1028F00001014051050DF350446B436F44C103F097
:102900004351F2CF43F1F29E000171EC00F0090057
:10291000F5CF03F0010143BFF28E416F03C042F1D6
:102920004CD001014051050DF350446B436F44C13D
:1029300003F04351F2CF43F1F29E000161EC00F04D
:102940000900F5CF03F0010143BFF28E416F03C0D0
:1029500042F133D001014051050DF350446B436FF8
:1029600044C103F04351F2CF43F1F29E000161EC08
:1029700000F00900F5CF03F0010143BFF28E416F73
:1029800003C042F11AD001014051050DF350446BD0
:10299000436F44C103F04351F2CF43F1F29E000173
:1029A00061EC00F00900F5CF03F0010143BFF28EA6
:1029B000416F03C042F101D0010141C101F042C1A8
:1029C00002F0000150EF15F0F2CF0EF0F29EE82475
:1029D000F76AF736ED0FF66E290EF7220A00F5506A
:1029E000FA6E0800F5500EBEF28EF96EF02822291C
:1029F00054298629010138C13BF1000B006E39C111
:102A000003F00050160E395D04E10052000109E0A8
:102A100001011A0E035C04E10052000128E00101EB
:102A20004DD001013A2D0DD03BC13FF10001AFDE89
:102A300001013D6B01C03CF1050E0001B86F0FD0E4
:102A40000101020E3A5D3E6F3BC13FF1406F000154
:102A5000BDD602C03DF101C03CF1060EB86F3CC1CD
:102A6000BDF000013DC1BEF00001010127D0010110
:102A70003A2D0ED03BC13EF100010DEC0FF00101EB
:102A80003D6B01C03CF1050E0001B86F0FD0010194
:102A9000020E3A5D3E6F3BC13FF1406F000120D70F
:102AA00002C03DF101C03CF1060EB86F3CC1BDF063
:102AB00000013DC1BEF00001010100D000014FDE68
:102AC00050EF17F0010142C1E9FF43C1EAFFEFCF28
:102AD00044F1030E4225E96E000E4321EA6EEFCF6A
:102AE00047F143C1EAFF42C1E9FF47C1EFFF030ECF
:102AF0004225E96E000E4321EA6E44C1EFFF010E4C
:102B00004225E96E000E4321EA6EEFCF44F1010E3B
:102B10004225016E000E4321036E020E4225E96E2E
:102B2000000E4321EA6EEFCF47F103C0EAFF01C078
:102B3000E9FF47C1EFFF020E4225E96E000E432177
:102B4000EA6E44C1EFFF010E4225456F000E43219E
:102B5000466F46C1EAFF45C1E9FFD890EF36446BA6
:102B6000D8B0442B42C145F143C146F1445302E180
:102B7000D89001D0D88046C1EAFF45C1E9FFEF36C1
:102B8000446BD8B0442B010E4225456F000E432103
:102B9000466F445302E1D89001D0D88046C1EAFF85
:102BA00045C1E9FFED320001000C330E486E010112
:102BB0002CC1E9FF2DC1EAFFEFCF31F1030E2C2527
:102BC000E96E000E2D21EA6EEFCF38F1020E2C25B2
:102BD000E96E000E2D21EA6EEFCF39F138C135F1E3
:102BE00039C134F1010E2C25E96E000E2D21EA6E5B
:102BF000EFCF33F135C139F134C138F13C6B2E6B75
:102C0000436B2EC142F1456B280E446F000187ECE7
:102C100002F002C03EF102C003F001010150F2CF08
:102C20003DF1F29E02C0F7FF000181EC00F00900C7
:102C3000F5CF03F001013DBFF28E3D6F03C03EF1C1
:102C40003D5302E13E532DE03C532BE1436B2EC13B
:102C500042F1456B280E446F000187EC02F002C080
:102C60003EF102C003F001010150F2CF3DF1F29EAE
:102C700002C0F7FF000181EC00F00900F5CF03F07E
:102C800001013DBFF28E3A6F03C03BF138513A5D0E
:102C900006E139513B5D03E1010E3C6F01D02E2B63
:102CA000AFD73CC101F00152D8B467EF1BF0436BC2
:102CB0002EC142F1456B280E446F000187EC02F0F3
:102CC00002C039F101C038F1030E01010124016E87
:102CD000000E0220036E0150F2CF38F1F29E03C0C5
:102CE000F7FF000181EC00F0010138BFF28E2F6F79
:102CF0002FC143F14351410A000113E0030A15E0DB
:102D0000010A17E0070A19E0010A1BE0030A1DE0A7
:102D1000010A1FE00F0A21E02B0A23E0030A25E045
:102D200028D0010E016E2BD02AD0010E016E27D0C3
:102D300026D0020E016E23D022D0040E016E1FD0C9
:102D40001ED0010E016E1BD01AD0020E016E17D0DC
:102D500016D0040E016E13D012D0040E016E0FD0E7
:102D60000ED0010E016E0BD00AD0020E016E07D0FC
:102D700006D0AA0E486E000E016E01D000D001C030
:102D800030F10101436B2EC142F1456B280E446FB7
:102D9000000187EC02F002C039F101C038F1020EE7
:102DA00001010124016E000E0220036E0150F2CFDA
:102DB00038F1F29E03C0F7FF000181EC00F0010141
:102DC00038BFF28E326F2F51610802E0000E01D041
:102DD000010E3011D8B464EF1BF04BC0B6F0000107
:102DE000050EB76F31C1B9F033C1BAF034C1BBF0D1
:102DF000000135C1BCF00001010131514008D8A4E7
:102E000003D2D20E486E333D2ED0010E2E25396FDF
:102E1000436B426F456B280E446F000187EC02F054
:102E200002C039F102C003F001010150F2CF38F1C4
:102E3000F29E02C0F7FF000181EC00F00900F5CF1F
:102E400003F0010138BFF28E346F03C035F134C195
:102E5000BDF0000135C1BEF00001060EB86F7FDC89
:102E6000486AD0D1010133530EE1060E0001B86F5C
:102E700001013251030B0001BD6F2FC1BEF06FDCA9
:102E8000486AC0D101012F5161080CE1D10E486E92
:102E900035C139F134C138F133C13AF10001AAD555
:102EA000B1D101013351F60847E2080E0001B86FB5
:102EB000F70E0101335D040DF3CF37F1040E366FC9
:102EC0003651070834E3036A3651030F016E000ED2
:102ED00003220150B60FE96E000E0320EA6E436B29
:102EE0002EC142F1456B280E446F000187EC02F0C1
:102EF00002C03BF101C03AF1060E01013A27000E73
:102F00003B2337513A25016E000E3B21036E0150E1
:102F1000F2CF3AF1F29E03C0F7FF000181EC00F01E
:102F200001013ABFF28EEF6E372B362BC9D7000165
:102F300016DC486A67D10101332D61D132A15FD11E
:102F4000396BBD0E386F2EC13AF12FC13BF13BC139
:102F500043F14351410A000113E0030A15E0010A5D
:102F600017E0070A19E0010A1BE0030A1DE0010A45
:102F70001FE00F0A21E02B0A23E0030A25E028D0F6
:102F8000010E016E2BD02AD0010E016E27D026D063
:102F9000020E016E23D022D0040E016E1FD01ED06F
:102FA000010E016E1BD01AD0020E016E17D016D082
:102FB000040E016E13D012D0040E016E0FD00ED08D
:102FC000010E016E0BD00AD0020E016E07D006D0A2
:102FD000AA0E486E000E016E01D000D001C03FF174
:102FE0000101436B3AC142F1456B280E446F000169
:102FF00087EC02F002C041F101C040F1020E010174
:103000000124016E000E0220036E0150F2CF40F148
:10301000F29E03C0F7FF000181EC00F0010140BF08
:10302000F28E800B800833E1436B3AC142F1456B6D
:10303000280E446F000187EC02F002C041F101C08C
:1030400040F1040E01010124016E000E0220036E06
:103050000150F2CF40F1F29E03C0F7FF000181EC76
:1030600000F00900F5CF03F0010140BFF28E3E6F82
:103070003EC140F139C142F138C141F13EC143F195
:103080003FC144F10001D7EC0CF036D00101436B95
:103090003AC142F1456B280E446F000187EC02F003
:1030A00002C041F101C040F1040E01010124016E92
:1030B000000E0220036E0150F2CF40F1F29E03C0D9
:1030C000F7FF000181EC00F00900F5CF03F00101EA
:1030D00040BFF28E3C6F03C03DF139C1EAFF38C1F9
:1030E000E9FF3DC1E2FF3CC1E1FF3F51016E04E059
:1030F000E6CFEEFF012EFCD701013B51480874E1F9
:1031000039C141F138C140F1010E4025436F000E35
:103110004121446F44C1EAFF43C1E9FFD890EF3633
:10312000426BD8B0422B40C143F141C144F14253FC
:1031300002E1D89001D0D88044C1EAFF43C1E9FF41
:10314000ED32426BD8B0422B010E4025436F000E8A
:103150004121446F425302E1D89001D0D88044C14C
:10316000EAFF43C1E9FFED3240C1E9FF41C1EAFF97
:10317000EFCF42F1030E4025E96E000E4121EA6EC9
:10318000EFCF45F141C1EAFF40C1E9FF45C1EFFF83
:10319000030E4025E96E000E4121EA6E42C1EFFFA9
:1031A000010E4025E96E000E4121EA6EEFCF42F19B
:1031B000010E4025016E000E4121036E020E4025D6
:1031C000E96E000E4121EA6EEFCF45F103C0EAFF40
:1031D00001C0E9FF45C1EFFF020E4025E96E000E78
:1031E0004121EA6E42C1EFFF000E016E040E302550
:1031F0000001B86FAFEC13F0486A04D00101AF0EC4
:10320000486E000162D2010131512008D8A45AD27F
:1032100032A353D2332D51D2040E2C25386F000E19
:103220002D21396F39C13BF138C13AF12EC13CF142
:103230002FC13DF13DC143F14351410A000113E06B
:10324000030A15E0010A17E0070A19E0010A1BE06A
:10325000030A1DE0010A1FE00F0A21E02B0A23E008
:10326000030A25E028D0010E016E2BD02AD0010ED2
:10327000016E27D026D0020E016E23D022D0040E7C
:10328000016E1FD01ED0010E016E1BD01AD0020E8F
:10329000016E17D016D0040E016E13D012D0040E9A
:1032A000016E0FD00ED0010E016E0BD00AD0020EAF
:1032B000016E07D006D0AA0E486E000E016E01D036
:1032C00000D001C040F101013D51480808E13BC177
:1032D00043F13AC142F1000162EC15F00101436B88
:1032E0003CC142F1456B280E446F000187EC02F0AF
:1032F00002C043F101C042F1020E01010124016E3E
:10330000000E0220036E0150F2CF42F1F29E03C084
:10331000F7FF000181EC00F0010142BFF28E800B4B
:10332000800833E1436B3CC142F1456B280E446F8A
:10333000000187EC02F002C043F101C042F1040E2B
:1033400001010124016E000E0220036E0150F2CF34
:1033500042F1F29E03C0F7FF000181EC00F009008A
:10336000F5CF03F0010142BFF28E416F41C142F13E
:103370003BC144F13AC143F141C145F140C146F17D
:103380000001A6EC05F037D00101436B3CC142F1CE
:10339000456B280E446F000187EC02F002C043F138
:1033A00001C042F1040E01010124016E000E022051
:1033B000036E0150F2CF42F1F29E03C0F7FF00010D
:1033C00081EC00F00900F5CF03F0010142BFF28E5D
:1033D0003E6F03C03FF13FC1EAFF3EC1E9FF3BC181
:1033E000E2FF3AC1E1FF4051016E04E0E6CFEEFF9B
:1033F000012EFCD70001000E016E0101396BBD0EDC
:10340000386F2EC13AF12FC13BF13BC143F143511B
:10341000410A000113E0030A15E0010A17E0070A58
:1034200019E0010A1BE0030A1DE0010A1FE00F0A70
:1034300021E02B0A23E0030A25E028D0010E016ECB
:103440002BD02AD0010E016E27D026D0020E016E9D
:1034500023D022D0040E016E1FD01ED0010E016EAB
:103460001BD01AD0020E016E17D016D0040E016EBA
:1034700013D012D0040E016E0FD00ED0010E016ECB
:103480000BD00AD0020E016E07D006D0AA0E486EED
:10349000000E016E01D000D001C03FF10101436B6D
:1034A0003AC142F1456B280E446F000187EC02F0EF
:1034B00002C041F101C040F1020E01010124016E80
:1034C000000E0220036E0150F2CF40F1F29E03C0C5
:1034D000F7FF000181EC00F0010140BFF28E800B8C
:1034E000800833E1436B3AC142F1456B280E446FCB
:1034F000000187EC02F002C041F101C040F1040E6E
:1035000001010124016E000E0220036E0150F2CF72
:1035100040F1F29E03C0F7FF000181EC00F00900CA
:10352000F5CF03F0010140BFF28E3E6F3EC140F186
:1035300039C142F138C141F13EC143F13FC144F1CB
:103540000001D7EC0CF036D00101436B3AC142F1D7
:10355000456B280E446F000187EC02F002C041F178
:1035600001C040F1040E01010124016E000E022091
:10357000036E0150F2CF40F1F29E03C0F7FF00014D
:1035800081EC00F00900F5CF03F0010140BFF28E9D
:103590003C6F03C03DF139C1EAFF38C1E9FF3DC1CD
:1035A000E2FF3CC1E1FF3F51016E04E0E6CFEEFFD8
:1035B000012EFCD701013B51480874E139C141F1AA
:1035C00038C140F1010E4025436F000E4121446F88
:1035D00044C1EAFF43C1E9FFD890EF36426BD8B04F
:1035E000422B40C143F141C144F1425302E1D89022
:1035F00001D0D88044C1EAFF43C1E9FFED32426BFC
:10360000D8B0422B010E4025436F000E4121446F7C
:10361000425302E1D89001D0D88044C1EAFF43C1AF
:10362000E9FFED3240C1E9FF41C1EAFFEFCF42F1CE
:10363000030E4025E96E000E4121EA6EEFCF45F101
:1036400041C1EAFF40C1E9FF45C1EFFF030E40253C
:10365000E96E000E4121EA6E42C1EFFF010E4025E6
:10366000E96E000E4121EA6EEFCF42F1010E4025D6
:10367000016E000E4121036E020E4025E96E000E20
:103680004121EA6EEFCF45F103C0EAFF01C0E9FF37
:1036900045C1EFFF020E4025E96E000E4121EA6EA2
:1036A00042C1EFFF000E016E040E30250001B86F1D
:1036B000AFEC13F0486A04D00101AF0E486E000170
:1036C00004D00101AE0E486E000103D00101AB0E23
:1036D000486E0001D5EF1EF001013F51FC0F65E27D
:1036E000040F0001DAEF1BF001014051050DF3500A
:1036F000436B426F020E4225016E000E4321036EA2
:103700000150F2CF42F1F29E00014FEC00F00101B6
:1037100042BFF28E416F49D001014051050DF35077
:10372000436B426F020E4225016E000E4321036E71
:103730000150F2CF42F1F29E000161EC00F0010174
:1037400042BFF28E416F31D001014051050DF3505F
:10375000436B426F020E4225016E000E4321036E41
:103760000150F2CF42F1F29E000161EC00F0010144
:1037700042BFF28E416F19D001014051050DF35047
:10378000436B426F020E4225016E000E4321036E11
:103790000150F2CF42F1F29E000161EC00F0010114
:1037A00042BFF28E416F01D0010141C101F0000121
:1037B0009DEF1CF0F2CF0EF0F29EE824F76AF73688
:1037C000D90FF66E370EF7220A00F550FA6E080090
:1037D000F5500EBEF28EF96EE83618374837783756
:1037E00001013F51FC0F79E2040F000174EF1CF05E
:1037F00001014051050DF350446B436F030E432507
:10380000016E000E4421036E0150F2CF43F1F29E8F
:1038100000014FEC00F00900F5CF03F0010143BFB8
:10382000F28E416F03C042F158D001014051050DA5
:10383000F350446B436F030E4325016E000E442189
:10384000036E0150F2CF43F1F29E000161EC00F0F3
:103850000900F5CF03F0010143BFF28E416F03C0B1
:1038600042F13BD001014051050DF350446B436FD1
:10387000030E4325016E000E4421036E0150F2CF6A
:1038800043F1F29E000161EC00F00900F5CF03F076
:10389000010143BFF28E416F03C042F11ED001010E
:1038A0004051050DF350446B436F030E4325016EE9
:1038B000000E4421036E0150F2CF43F1F29E00014D
:1038C00061EC00F00900F5CF03F0010143BFF28E77
:1038D000416F03C042F101D0010141C101F042C179
:1038E00002F00001A4EF1CF0F2CF0EF0F29EE824EB
:1038F000F76AF7360D0FF66E390EF7220A00F5500B
:10390000FA6E0800F5500EBEF28EF96EF0372A38C6
:1039100064389E382EC13FF1C7EC13F001C03AF174
:1039200001013C6B3B6B3A513B5DD8B0CFD02EC10F
:103930003FF13BC140F10001CFD601C03DF12EC1A6
:103940003FF13BC140F14CD702C040F101C03FF113
:10395000036A01013C512C25416F2D510320426F18
:103960003DC143F14351410A000113E0030A15E050
:10397000010A17E0070A19E0010A1BE0030A1DE02B
:10398000010A1FE00F0A21E02B0A23E0030A25E0C9
:1039900028D0010E016E2BD02AD0010E016E27D047
:1039A00026D0020E016E23D022D0040E016E1FD04D
:1039B0001ED0010E016E1BD01AD0020E016E17D060
:1039C00016D0040E016E13D012D0040E016E0FD06B
:1039D0000ED0010E016E0BD00AD0020E016E07D080
:1039E00006D0AA0E486E000E016E01D000D001C0B4
:1039F00043F140C1EAFF3FC1E9FF42C1E2FF41C1DB
:103A0000E1FF01010150016E04E0E6CFEEFF012E5F
:103A1000FCD73D5148080EE1036A3C512C253F6F0D
:103A20002D510320406F436F3FC142F1000162EC12
:103A300015F001013DC143F14351410A000113E07A
:103A4000030A15E0010A17E0070A19E0010A1BE062
:103A5000030A1DE0010A1FE00F0A21E02B0A23E000
:103A6000030A25E028D0010E016E2BD02AD0010ECA
:103A7000016E27D026D0020E016E23D022D0040E74
:103A8000016E1FD01ED0010E016E1BD01AD0020E87
:103A9000016E17D016D0040E016E13D012D0040E92
:103AA000016E0FD00ED0010E016E0BD00AD0020EA7
:103AB000016E07D006D0AA0E486E000E016E01D02E
:103AC00000D0015001013C273B2B2DD70001000CF9
:103AD000959A8C7A140EFB25E96E000EFC21EA6E95
:103AE0003E50EF6E150EFB25E96E000EFC21EA6ECE
:103AF0003DC0EFFF090EFB25E96E000EFC21EA6ECA
:103B00003FC0EFFF020E01012C6F090E0001FB25E3
:103B1000E96E000EFC21EA6E020EEF2401012C5D1D
:103B200028E2036A2C51140F016E000E032201508B
:103B30000001FB25016EFC51032201C02DF10101A2
:103B400003C02EF1020E2C5D036A030F016E000EFE
:103B5000032201503D0FE96E000E0320EA6EEFCF05
:103B60002FF12EC1EAFF2DC1E9FF2FC1EFFF2C2B52
:103B7000CCD7010E0001FB25E96E000EFC21EA6E98
:103B8000010EEF6E12EF1FF0D650D7CF03F00101F8
:103B90002C6FD7502D6F4B0832E2FF0A03E12C51F6
:103BA00047082DE2959C8C7C76CF36F075CF37F0A8
:103BB00048C038F0EA6A390EE96EE26ACF0EE16E6B
:103BC000020E016EE6CFEEFF012EFCD733C03FF1AF
:103BD00032C03EF1020E406F426B350E416F34C071
:103BE00043F1FC0E446F000134EC08F0D66B010E7B
:103BF000D56FD76AD66A016E06D005D00101000ED6
:103C0000016E000100D015EF1FF001012C6B2C514B
:103C1000030863E3036A2C512E0FE96E000E0320A4
:103C2000EA6EEF5256E02C510B0DF3502E6B2D6FB8
:103C30005E0E2D25E96E000E2E21EA6EECCF2EF1E0
:103C4000ED52EFCF2DF12C51010B2F6F2C510B0D9D
:103C5000F350316B306F030E3025016E000E3121B1
:103C6000036E01505E0F016E000E032201C030F1A1
:103C700003C031F12C510B0DF350336B326F020E38
:103C80003225016E000E3321036E01505E0FE96E86
:103C9000000E0320EA6EEFCF32F12EC13FF12DC1AD
:103CA0003EF12FC140F131C142F130C141F132C189
:103CB00043F1FC0E446F000134EC08F001520AE0BD
:103CC000036A01012C512E0FE96E000E0320EA6EEB
:103CD000EF6A000101012C2B9AD7000E016E000142
:103CE0001AEF1FF001012A6B2D6B3D0E2C6F2F6B0D
:103CF000400E2E6F316B3F0E306F010E336F2B0E67
:103D0000326F000133EF12F00152D8B48BD0010EA4
:103D100001012A6F4A2A2B51600B04E02B51600BE2
:103D2000486E81D02BA701D0492A340E486E3D52EF
:103D300023E13E5221E14B50415C02E0415217E148
:103D40004050010A000105E0030A06E0830A07E08B
:103D500009D0050E356E09D0040E356E06D085ECFF
:103D60000EF003D0CC0E486E00D004D00101CD0E71
:103D7000486E000157D001014BC001F0060E036EE2
:103D80004B503D5C14E103503E5C11E13F50030891
:103D900009E22D6B400E2C6F0001D5EF15F00001EC
:103DA00004D00101A90E486E00013CD0010135503C
:103DB000050839E100018A513D5C0BE18B513E5C05
:103DC00008E101012D6B400E2C6F2E6B0001A2DD6E
:103DD00029D095513D5C0CE196513E5C09E1010111
:103DE0002D6B400E2C6F010E2E6F000193DD1AD04B
:103DF000A0513D5C0CE1A1513E5C09E101012D6B3C
:103E0000400E2C6F020E2E6F000184DD0BD03DC0E2
:103E10002CF101012D6B4C503D5C05E12D5303E16C
:103E2000000156D601010001AFD6015001012A134D
:103E30000001EBD6015001012A132AC101F0000153
:103E4000E3EF21F001012B512D19800B2F6F2BAFC8
:103E500005D02A1F2B1F2A2BD8B42B2B2DAF05D012
:103E60002C1F2D1F2C2BD8B42D2B016A026A006A3F
:103E7000036A2D5102E12C5118E0100E2E6FD890DC
:103E80002A372B37003603362D51035C02E12C51C3
:103E9000005C07E32C51005ED8A003062D51035EA1
:103EA000D880013602362E2FEAD72FAF05D0011E5B
:103EB000021E012AD8B4022A0001000C640E01017E
:103EC0002A252C6F010E2D6FD8B02D2B2B512C25B0
:103ED000086F0851FF0A010F086FAC8A800E2C6F23
:103EE0000001AFEC0EF0E40E01012C6F0001AFEC0D
:103EF0000EF02AC12CF1AFEC0EF02BC12CF1AFEC7F
:103F00000EF008C12CF1AFEC0EF0AC9A000C660E6E
:103F100001012A252C6F010E2D6FD8B02D2B2B51AE
:103F20002C25086F0851FF0A010F086FAC8A800E1C
:103F30002C6F0001AFEC0EF0E60E01012C6F0001BA
:103F4000AFEC0EF02AC12CF1AFEC0EF02BC12CF12E
:103F5000AFEC0EF008C12CF1AFEC0EF0AC9A000CF7
:103F60006F0E0101086F0851FF0A010F086FAC8A3C
:103F7000800E2C6F0001AFEC0EF0EF0E01012C6FE4
:103F80000001AFEC0EF001012C6B0001AFEC0EF064
:103F900001012C6B0001AFEC0EF008C12CF1AFEC6D
:103FA0000EF0AC9A0DEF21F001012E51D8B471D072
:103FB000006E3251D8B46DD0002604E3810E002685
:103FC00068E204D07F0E005E64E363E02FC136F147
:103FD0003351361B2F8F338F31513503F4CF38F1E6
:103FE00030513403F4CF03F0F3CF37F13503F350FE
:103FF0003827F4503723000E032231513403F35095
:104000003827F4503723000E026A032202222F5170
:104010003503F3503727F4500322000E02222F51AC
:104020003403F3500326F4500222000E016A0122E9
:1040300031513303F3503727F4500322000E02228C
:10404000012230513303F3500326F4500222000EB4
:1040500001222F513303F3500226F4500122002A8B
:1040600001BE05D037370336023601360006000E92
:1040700037AF0AD0032A02220122015005E1025083
:1040800003E1035001E1002A36BF018E36AF019EE5
:1040900004D0006A016A026A036A000133EF21F06A
:1040A0008E0E006E01012A51005E2BC102F02CC160
:1040B00001F0028E005209E0D890025202E1015252
:1040C00004E002320132002EF7D72BAF05D0011EDB
:1040D000021E012AD8B4022A00013CEF21F0D45379
:1040E000D8B478D0D15101011E5D05E10001D25153
:1040F00001011F5D48E0D2C01FF1D1C01EF10001D7
:10410000D2BF08D0D251220805E2FF0A3BE1D151CB
:10411000280838E3D2AF07D0D251DC0804E332E1FB
:10412000D151D7082FE2D2C025F1D1C024F1A40E7D
:1041300001012425206F380E2521216F21C12BF18B
:1041400020C12AF12D6B0A0E2C6F00017BDE02C00C
:1041500021F101C020F1010121C122F120C123F18F
:10416000860E2A6FD3C02BF10001A8DEC30E010119
:104170002A6FD3C02BF10001A1DE22C12AF123C195
:104180002BF1C5DE0101D650D7CF03F02A6FD7CF70
:104190002BF127C143F126C142F1D6C045F1D5C06C
:1041A00044F1000187EC02F00250036E01012B5D27
:1041B0000FE303E101502A5D0BE30001DFEC0EF099
:1041C00002C0DAF001C0D9F0D52BD8B4D62B01014A
:1041D00087D00001D15101011C5D06E10001D251DF
:1041E00001011D5DD8B47CD0D2C01DF1D1C01CF13D
:1041F0000001D2BF08D0D251220805E2FF0A0CE12B
:10420000D151280809E3D2AF0FD0D251DC080CE31A
:1042100003E1D151D70808E3A3D6140E01012E6F94
:10422000000173EC02F05BD0D2C02DF1D1C02CF1B3
:10423000F7EC0CF000C02AF101C02BF102C02CF108
:1042400003C02DF103C031F102C030F101C02FF1E4
:1042500000C02EF112C135F111C134F110C133F19A
:104260000FC132F1A1D603C02DF102C02CF101C063
:104270002BF100C02AF114D7015001011325246F3E
:1042800002501421256FA40E2425206F380E2521FD
:10429000216F21C12BF120C12AF12D6B0A0E2C6F49
:1042A0000001D0DD02C021F101C020F1010121C1D6
:1042B00022F120C123F1860E2A6FD3C02BF1000119
:1042C000FDDDC30E01012A6FD3C02BF10001F6DD25
:1042D00022C12AF123C12BF11ADE959E8C7E0101A9
:1042E000C282C2B2FED7C3CFDBF00001E4EF21F0FF
:1042F000F86AD09E088EEA6AE96AB896400EAF6EF8
:10430000A60EAC6E900EAB6E9488949A94968B9693
:1043100093908A80C150C00B0F09C16E070EB46E16
:104320004B6A4C6AD16BD26B010ED56FD66BD76BD3
:10433000D86BD96BDA6BDB6BDC6BFC6BDD0EFB6F68
:104340000101066B0791450E0D6F010E0E6F1C6B80
:104350001D6B1E6B1F6B266B276B959E8C9E000141
:1043600043EF02F085EC0EF04AEC09F0D650D7CFBF
:1043700003F001012A6FD7CF2BF1D8C043F1D7C08A
:1043800042F1D6C045F1D5C044F1000187EC02F0FE
:104390000250036E01012B5D14E303E101502A5D1D
:1043A00010E30001CD5305E1CE53D8A402D00101A2
:1043B00008D00101066B000113EF12F0D52BD8B421
:0C43C000D62B00018FD48BD6CFD7030082
:020000040030CA
:0E00000000021F1E008281000FC007E00740B3
:00000001FF
